:0600000002117702006B03
:03000B0002006B85
:0300130002006B7D
:03001B0002006B75
:0300230002006B6D
:03002B0002006B65
:0300330002006B5D
:03003B0002006B55
:0300430002006B4D
:03004B0002006B45
:0300530002006B3D
:03005B0002006B35
:0300630002006B2D
:01006B003262
:1000800002006B0002006B0002006B0002006B00BC
:1000900002006B0002006B0002006B0002006B00AC
:1000A00002006B0002006B0002006B0002006B009C
:0800B00002006B0002006B006E
:1001000002006B0002006B0002006B0002006B003B
:1001100002006B0002006B0002006B0002006B002B
:1001200002006B0002006B0002006B0002006B001B
:1001300002006B0002006B0002006B0002006B000B
:1001400002006B0002006B0002006B0002006B00FB
:1001500002006B0002006B0002006B0002006B00EB
:1001600002006B0002006B0002006B0002006B00DB
:1001700002006B0002006B0002006B0002006B00CB
:10018000438080C28122C01A85811AAA8253807F4F
:10019000E51A24FBF88682C002120277D002E51A23
:1001A00024FCF8746056FB602CBB20028005BB4029
:1001B0001F800CA81A181818868212027780168AD7
:1001C00082120277A81A1818188682120277800500
:1001D0007582018025E51A24F8F8E66017E51A24EF
:1001E000F8F8E6C0E0E51A24F9F88682088683125A
:1001F000033B1581438080758200D01A22C01A8586
:10020000811AAA8253807FE51A24FBF88682C002F5
:10021000120277D002E51A24FCF8746056FB602FB6
:10022000BB20028005BB401F800CA81A1818188636
:100230008212027780198A82120277A81A18181877
:10024000868212027780084380807582018025E5CE
:100250001A24F8F8E66017E51A24F8F8E6C0E0E595
:100260001A24F9F886820886831202C81581438011
:1002700080758200D01A22E58223FA139281D280FF
:10028000C280EA23FA139281D280C280EA23FA1351
:100290009281D280C280EA23FA139281D280C280F6
:1002A000EA23FA139281D280C280EA23FA13928160
:1002B000D280C280EA23FA139281D280C280EA23DC
:1002C000139281D280C28022C01A85811AAA82AB81
:1002D00083A81A18181886048C051CED601E8A82E3
:1002E0008B83E0FDA3AA82AB838D82C002C003C0D2
:1002F00004120277D004D003D00280DCD01A22E4AA
:10030000D280A28333C280D280A28333C280D280C3
:10031000A28333C280D280A28333C280D280A283E0
:1003200033C280D280A28333C280D280A28333C200
:1003300080D280A28333C280F58222C01A85811ABE
:10034000AA82AB83A81A18181886048C051CED60C5
:10035000121202FFAD828A828B83EDF0A3AA82ABD8
:060360008380E8D01A22A0
:03117D00021185D7
:03119800021180C1
:0511800012084480FE8E
:10036600C200E4F508F509F50AD201750B00750C13
:1003760000120A29120A2675CB6375CAC0758E004B
:1003860075C804D2AFD2B0D2B190E60B7403F000B8
:1003960090E6047480F00090E6047402F00090E6A3
:1003A600047404F00090E6047406F00090E6047409
:1003B60008F00090E604E4F00090E61074A0F00067
:1003C60090E61174A0F00090E618E4F00090E612B2
:1003D60074A2F00090E619E4F00090E61374A0F021
:1003E6000090E60BE4F00090E61474A2F00090E6AC
:1003F6001AE4F00090E61A7411F00090E61574E025
:10040600F00090E61BE4F00090E61B7409F0009003
:10041600E626E4F00090E6277440F00090E691743A
:1004260080F00090E6957480F00090E6917480F07C
:100436000090E6957480F00043A08090E6FBE054BF
:10044600FDF022AA82850C827583E0EAF0050C0590
:1004560009E4B50902050A22C01AE581F51A240441
:10046600F581200003020626120A2590E6A2E0FA8C
:1004760030E103020502E509450A60687AC07BE7B8
:100486008B9D7AC07BE77B008A9E90E67C7431F078
:100496007460F0C3743E9509E4950A50107A3EE5FF
:1004A6000924C2F509E50A34FFF50A8007AA09E41A
:1004B600F509F50A8A037C007DE08D9A850B9B8AF7
:1004C600041AEC601090E67BE090E67CF07C007D00
:1004D600E08D9A80EA859B0B0090E68F74022BF0E4
:1004E600D2CF801830CF1590E7C07431F090E7C1B5
:1004F6007460F00090E68F7402F0C2CFE5AA30E097
:1005060003020626C3E50994C1E50A9400400302E6
:10051600062690E690E0FB7A0090E691E07D0042A8
:1005260002ED4203A81A080808A60208A6037C00E2
:100536007DF08D9A7C007DF07D008C9BA81A08E4E6
:10054600F608F6A81A08A91A090909C3E69708E6DB
:100556000997400302061FE50870030205E7A81A7B
:10056600080808A91A09E6C397FE08E60997FFAA2C
:10057600087B00C3EA9EEB9F50048A068B078E0217
:10058600E508C39AF508A81A08EE26F6EF0836F627
:100596003001248E028F038A048B051ABAFF011BD1
:1005A600EC4D609F90E67BE0F582C002C003120A24
:1005B60067D003D00280E08E028F038A048B051A6F
:1005C600BAFF011BEC4D700302054990E67BE0F58E
:1005D60082C002C003120AA4120449D003D00280CA
:1005E600DA90E67BE0FA23235401FBB40100920182
:1005F600EA30E707743F5AF50880123001078A820D
:10060600120A4380088A82120A59120449A81A0853
:1006160006B6000208060205490090E6917480F0CD
:10062600851A81D01A2290E6B8E0FA20E75F90E6B4
:10063600B9E07002D20090E6B9E0FABA994B90E6BA
:100646008BE4F090E6A0E0FA20E1F890E6BCE0FA50
:1006560090E6BDE0FB90E6BAE0FC90E6BBE0FD90DC
:10066600E68BE0C0E07440C0E074E7C0E0C002C0C2
:1006760003C0048D821201FDAA82E58124FAF58168
:10068600EAB40100E433F582227582012290E6B9CC
:10069600E0FABA911C90E6BCE0700C90E6FBE054E0
:1006A600FDF0120B36800A90E6FBE04402F0120BD6
:1006B6003690E6B9E0FABA920E90E6BCE0700543D1
:1006C600A080800353A07F90E6B9E0FABA931A900F
:1006D600E601E0FA30E30A90E601E0FA54F7F0802A
:1006E6000890E601E0FA4408F090E6B9E0FABA9418
:1006F6000890E601E0FA54F7F090E6B9E0FABA9607
:100706000F43B28B12018090E740E4F090E741F08E
:1007160090E6B9E0FABA972C53B27490E740744267
:10072600F090E7417443F090E7427442F090E7435B
:100736007443F090E68AE4F090E6BEE090E68BF033
:100746007582012290E6B9E0FABA984E90E6BEE0CC
:10075600FA90E6BCE0FB90E6BDE0FC90E6BAE0FD70
:1007660090E6BBE0FEC0027440C0E074E7C0E0C0A3
:1007760003C004C0058E82120186AA82E58124FA8E
:10078600F581EA60047582002290E68AE4F090E63C
:10079600BEE090E68BF07582012290E6B9E0FABAE7
:1007A600953153807F90E6BAE0F58212027790E6A3
:1007B600BCE0F5821202771202FFAA8290E740EAB5
:1007C600F043808090E68AE4F090E68B7401F07541
:1007D60082012290E6B9E0FABA902B90E6BCE025B9
:1007E600E0547FFA2400F582E43418F583E0FB90A8
:1007F600E740F0EA042400F582E43418F583E0FAD1
:1008060090E741F0800C90E7407436F090E7417431
:1008160083F090E68AE4F090E6BEE0FABA02005071
:100826000790E6BEE0FA80027A0290E68BEAF0755F
:10083600820122300203120CD712045E80F5C2AF89
:100846001203661208A01210AA120C41D2AF120BA4
:040856003602083925
:10E100001201100100000040FB090160000401023F
:10E1100003010A061001FFFFFF400100090237005A
:10E12000020100804B0904000002FFFFFF02070507
:10E1300081024000000705020240000009040100BE
:10E1400002FFFFFF02070506020002000705880222
:03E15000000200CA
:10E154001201100100000040FB09016000040102EB
:10E1640003010A061001FFFFFF4001000902370006
:10E17400020100804B0904000002FFFFFF020705B3
:10E18400810240000007050202400000090401006A
:10E1940002FFFFFF02070506024000000705880290
:10E1A40040000003AEE1B4E1C2E10603000009044B
:10E1B4000E0341006C0074006500720061001803D6
:10E1C4005500530042002D0042006C0061007300B2
:10E1D400740065007200120330003000300030001B
:08E1E400300030003000300073
:10085A00AA82E50D54FEFBB50D0280298A048C0597
:10086A00E4620EED620FEB2400F582E43418F5839E
:10087A00E0FB7C00620EEC620FE50E33C50F33C558
:10088A000F92E0F50EAB0D050DEB2400F582E43472
:10089A0018F583EAF022750D00750EAA750FAA7570
:1008AA00820012085A75820012085A7A00C3EA6452
:1008BA008094865017EA2408F582E434E1F583E04F
:1008CA00F582C00212085AD0020A80E17A00C3EA0D
:1008DA00648094825017EA2423F582E434E1F58394
:1008EA00E0F582C00212085AD0020A80E175821C21
:1008FA0012085A75820012085A7A00C3EA64809470
:10090A00825017EA2402F582E434E1F583E0F582A5
:10091A00C00212085AD0020A80E17486250DFAF53F
:10092A0082C00212085A90E1B4E0F58212085AD045
:10093A000290E1B4E02AFAF582C00212085A90E164
:10094A00C2E0F58212085AD00290E1C2E02AF5828A
:10095A0012085A90E1DAE0F58212085A7A0090E118
:10096A00B4E0FBC3EA64808BF063F08095F0501723
:10097A00EA24B4F582E434E1F583E0F582C0021298
:10098A00085AD0020A80D77A0090E1C2E0FBC3EA93
:10099A0064808BF063F08095F05017EA24C2F582E8
:1009AA00E434E1F583E0F582C00212085AD0020A63
:1009BA0080D77A0090E1DAE0FBC3EA64808BF063C7
:1009CA00F08095F05017EA24DAF582E434E1F583F1
:1009DA00E0F582C00212085AD0020A80D77A00C310
:1009EA00EA648094845017EA240EF582E434E1F52F
:1009FA0083E0F582C00212085AD0020A80E17482AA
:100A0A00250D400875820012085A80F2AA0E901825
:100A1A007EEAF0AA0F90187FEAF022222222229080
:100A2A00E6007412F090E6017403F0AAB574FD5A58
:100A3A00F5F0748D45F0F5B522E582FA1392B2EA23
:100A4A00A2E192B1EAA2E492B3EAA2E592B4221236
:100A5A000A43A2B0E433FA74024AF58222E5821309
:100A6A0092B3D2B213C2B292B3D2B213C2B292B397
:100A7A00D2B213C2B292B3D2B213C2B292B3D2B248
:100A8A0013C2B292B3D2B213C2B292B3D2B213C2E7
:100A9A00B292B3D2B200C2B22222E582A2B01392BB
:100AAA00B3D2B2C2B2A2B01392B3D2B2C2B2A2B09D
:100ABA001392B3D2B2C2B2A2B01392B3D2B2C2B23A
:100ACA00A2B01392B3D2B2C2B2A2B01392B3D2B24C
:100ADA00C2B2A2B01392B3D2B2C2B2A2B01392B34C
:100AEA00D2B2C2B2F58222227880E84400600C7940
:100AFA0001901800E4F0A3D8FCD9FAD083D082F68A
:100B0A00D8FDC082C0837582002290E6A0E044012D
:100B1A00F022AA8274805AC423541FFB740F5A907D
:100B2A00E6834BF090E683E04420F02290E680E0F2
:100B3A00440AF09000FA12116690E65D74FFF09094
:100B4A00E65F74FFF05391EF90E680E054F7F022ED
:06119200E478FFF6D8FD31
:0611770075100075110067
:100B5A0090E680E0FA30E7267512007513E1751405
:100B6A00127515E175161C7517E17518707519E17E
:100B7A0090E6267402F00090E627E4F0002275124F
:100B8A00547513E17514667515E17516707517E1DC
:100B9A0075181C7519E190E626E4F00090E62774B2
:100BAA0040F000225391EF75A100D20232C021C059
:100BBA00E0C0F0C082C083C002C003C004C005C048
:100BCA0006C007C000C001C0D075D0005391EF75B0
:100BDA00A100120B5AD0D0D001D000D007D006D035
:100BEA0005D004D003D002D083D082D0F0D0E0D098
:100BFA002132C021C0E0C0F0C082C083C002C0035D
:100C0A00C004C005C006C007C000C001C0D075D06E
:100C1A00005391EF75A100120B5AD0D0D001D00029
:100C2A00D007D006D005D004D003D002D083D0821A
:100C3A00D0F0D0E0D02132120B5A751BAE751C0BC6
:100C4A00758200121003751BB7751C0B7582101282
:100C5A001003751BFC751C0B75821412100390E6A9
:100C6A005C7431F022E582547FFA24F750047582CD
:100C7A000022BA010475820122530201E4BA00017A
:100C8A0004F58222AA82BA010C90E6A1E0FB7C005C
:100C9A008B828C8322BA810C90E6A2E0FB7C008BCB
:100CAA00828C832253027FEA700C90E6A0E0FB7CE0
:100CBA00008B828C832290E6A3E0FB7C00EAC313BC
:100CCA00FA7D00EA2BFBED3C8B82F58322C202906F
:100CDA00E6B8E0FA530260BA00028028BA2002801D
:100CEA000DBA4002800EBA60028003020F98120BFE
:100CFA0014020F9812062CE5826003020F98120B59
:100D0A0014020F9890E6B8E0FA530280BA80028083
:100D1A0003020E9690E6B9E0FABA0003020E0FBA81
:100D2A0006028035BA08028008BA0A028017020E43
:100D3A009090E740E510F090E68AE4F090E68B7434
:100D4A0001F0020F9890E740E511F090E68AE4F08E
:100D5A0090E68B7401F0020F9890E6BBE0FABA01B4
:100D6A00028017BA02028038BA03028059BA060210
:100D7A00801BBA0702803C020E09AA12AB1390E646
:100D8A00B3EBF07B0090E6B4EAF0020F98AA14AB3A
:100D9A001590E6B3EBF07B0090E6B4EAF0020F9808
:100DAA00AA16AB1790E6B3EBF07B0090E6B4EAF034
:100DBA00020F98AA18AB1990E6B3EBF07B0090E605
:100DCA00B4EAF0020F9890E6BAE0FA90E1A7E0FBE5
:100DDA00C3EA9B4006120B14020F9890E6BAE0751C
:100DEA00F002A424A8F58274E135F0F583E0FAA3B1
:100DFA00E090E6B3F07B0090E6B4EAF0020F9812B6
:100E0A000B14020F9890E6B8E0FA53021FBA0002D8
:100E1A00800ABA0102801BBA0266802C90E740E47D
:100E2A00F090E741F090E68AF090E68B7402F002C7
:100E3A000F9890E740E4F090E741F090E68AF0904E
:100E4A00E68B7402F0020F9890E6BCE0F582120C71
:100E5A006FE582602590E6BCE0F582120C8EE0FA1E
:100E6A0053020190E740EAF090E741E4F090E68A05
:100E7A00F090E68B7402F0020F98120B14020F988E
:100E8A00120B14020F98120B14020F9890E6B9E095
:100E9A00FA24F45003020F95EA2A2A900EA9730243
:100EAA000F95020EE2020F5D020F3E020F95020F2E
:100EBA0095020F95020F95020F95020ECD020F951E
:100ECA00020ED953B1BF90E6BAE0F510020F98901E
:100EDA00E6BAE0F511020F9890E6B8E0FA53021F5D
:100EEA00BA00028005BA0247800A90E6BAE0120BFD
:100EFA0014020F9890E6BAE0703090E6BCE0F582F2
:100F0A00120C6FE582602390E6BCE0F582120C8E2B
:100F1A00AA82AB83E0FC5304FE8A828B83ECF090B6
:100F2A00E6BCE0F582120B1C8064120B14805F127F
:100F3A000B14805A90E6B8E0FA53021FBA004F9099
:100F4A00E6BAE0FABA01028005BA02028040120B40
:100F5A0014803B90E6BAE0FA702C90E6BCE0F58289
:100F6A00120C6FE582601A90E6BCE0F582120C8ED4
:100F7A00AA82AB83E0FC4304018A828B83ECF08073
:100F8A000D120B148008120B148003120B1490E636
:100F9A00A0E04480F022AA82BA03004005EA249C19
:100FAA00500122740F5AFBBB03028007740F5AFBCD
:100FBA00BB0B45A2AF9203C2AFEA2400F582E43428
:100FCA0000F5837402F07B0074012AFCE43BFDEC1B
:100FDA002400F582ED3400F583E51CFCF074022A46
:100FEA00FAE43BFBEA2400F582EB3400F583AA1B02
:100FFA007B00EAF0A20392AF22E582FA2483500131
:10100A0022EA5403600122A2AF9204C2AFEA24008A
:10101A00F582E43401F5837402F07B0074012AFC42
:10102A00E43BFDEC2400F582ED3401F583E51CF088
:10103A0074022AFAE43BFBEA2400F582EB3401F558
:10104A0083AA1BEAF0A20492AF22AA82BA800040C5
:10105A0005EA244B500122EA5403600122A2AF920E
:10106A0005C2AFEA2480F582E43400F5837402F005
:10107A007B0074012AFCE43BFDEC2480F582ED340C
:10108A0000F583E51CF074022AFAE43BFBEA2480AB
:10109A00F582EB3400F583AA1BEAF0A20592AF228F
:1010AA00C2E8C2EA751B00751C01758243120FA0C3
:1010BA00751B80751C00758253120FA00090E650B4
:1010CA00E4F00090E652E4F00090E654E4F0009078
:1010DA00E656E4F00090E65174FFF00090E653748F
:1010EA00FFF00090E65574FFF00090E65774FFF0A9
:1010FA000090E658E4F090E65974FFF090E65AE45E
:10110A00F090E65B74FFF090E65CE4F090E65D74C4
:10111A00FFF090E65EE4F090E65F74FFF00090E680
:10112A0060E4F00090E66174FFF090E662E4F0900B
:10113A00E66374FFF090E665E4F090E668740BF0FD
:10114A005391AFD2E8D2EA2222AA82121152DAFBD2
:10115A002290FB50A3E582458370F922AA82AB83D1
:0D116A0012115B1ABAFF011BEA4B70F42250
:0D118500758121120AF2E5826003021180DB
:00000001FF
